:020000040000FA
:10000000000001308A003429F300030E8301F4005C
:100010000408F700DD180E280B18162875080C05C3
:10002000F60076191429F61A1C292D292330F2001E
:10003000851620305C18183E8400DC1C2728D70B5E
:100040002528253080006308D70029230C293C236C
:1000500072088000840AD4015E1C4B28B2309300E1
:100060008C1D30288C1193008C1D34288C111308A2
:10007000D4078000840A93008C1D3C288C1113083F
:10008000D4078000840A93008C1D44288C11130827
:10009000D4078000840ADE1C6A28B03093008C1DCF
:1000A0004F288C1193008C1D53288C111308D407F2
:1000B0008000840A93008C1D5B288C111308D407E0
:1000C0008000840A93008C1D63288C111308D407C8
:1000D0008000840A5E1D8928B13093008C1D6E2833
:1000E0008C1193008C1D72288C111308D40780008A
:1000F000840A93008C1D7A288C111308D407800081
:10010000840A93008C1D82288C111308D407800068
:10011000840ADE1DA828B43093008C1D8D288C1114
:1001200093008C1D91288C111308D4078000840A39
:1001300093008C1D99288C111308D4078000840A21
:1001400093008C1DA1288C111308D4078000840A09
:100150005E1EC728B53093008C1DAC288C1193000F
:100160008C1DB0288C111308D4078000840A9300DA
:100170008C1DB8288C111308D4078000840A9300C2
:100180008C1DC0288C111308D4078000840ADE1E41
:10019000E628B63093008C1DCB288C1193008C1D63
:1001A000CF288C111308D4078000840A93008C1D7B
:1001B000D7288C111308D4078000840A93008C1D63
:1001C000DF288C111308D4078000840A5E1F0529DC
:1001D000B73093008C1DEA288C1193008C1DEE28FB
:1001E0008C111308D4078000840A93008C1DF62814
:1001F0008C111308D4078000840A93008C1DFE28FC
:100200008C111308D4078000840A5408D900D90936
:10021000D90A59088000DC148512DD18F5298B11E4
:1002200006080B108B152D29D6038E018F010C119A
:10023000560803195B152D291A08243C031D2C2987
:10024000D301F122F000F1225308031D2C2970087C
:10025000D33A031D2C29DB142D2977088400740E52
:100260008300F30E730E09008316031320309400ED
:1002700083120313203094007008D13A03195129D6
:100280007008B33A03191F2A7008B53A03191D2ADA
:100290007008D83A0319692A7008D93A0319892ACB
:1002A000CB2A831203178F011830CE22E100611888
:1002B0008510611C8514E1180511E11C05156119F3
:1002C0000811611D0815E1198811E11D8815611AD1
:1002D0008515611E8511E11A8610E11E0611203078
:1002E000CE22DD002230CE22DE002330CE22DF00FF
:1002F0002430CE22303090002530CE22950026309A
:10030000CE2296002730CE22E2002830CE22E30013
:100310002930CE22E400E40A4F23D5018030D600F4
:100320003C23560893008C1D93298C11D60A55083E
:10033000CE2293008C1D9A298C11D50A5508CE2205
:1003400093008C1DA1298C11D50A5508CE2293004B
:100350008C1DA8298C11D50A5608803A083C031D2B
:10036000902946236308D700D301D4010A309700AF
:100370008C016208D6008E018F012030F500DD1857
:1003800075157508831603138C000113831203136C
:10039000C0308B005D1CD2298B1106080B108B1509
:1003A0005823DE29DD1CD7291014DB11DE295D1D41
:1003B0000D2A8B1106080B108B154623DB180D2A0E
:1003C000DD1CF5295B1DDE295B116208D600582370
:1003D000DB19ED29E40BDE29DB15E11AF229061AF7
:1003E000EF291628861AF2291628DC1CDE295C1C47
:1003F000FB295C10FC295C14DC1020305C1C183ECE
:1004000084005F08D5008718032A0C1E052A0008FF
:100410009900840AD50B032ADE2910108B0183165C
:1004200003138C0183120313DB106123061586145A
:100430008511D430F1001423CB2AE116202AE112D1
:1004400006158614E11A8610E11E0611E2223A3CD6
:10045000031D682AD301F122D800F1225308031D9D
:10046000682A0230D5003C23803093008C1D362A48
:100470008C11580893008C1D3B2A8C11FE30930080
:100480008C1D402A8C11580893008C1D452A8C1114
:100490003C23B33093008C1D4B2A8C1193008C1D90
:1004A0004F2A8C1193008C1D532A8C1193008C1DA4
:1004B000572A8C1113085802031D682AD50B612A8C
:1004C000632AD809332A06158614B430F1001423A0
:1004D000CB2AD3018312031707308F00FF308D0022
:1004E0001F232130E922831203170E0883120313FE
:1004F000D307D9000323831203170C0883120313B5
:10050000D307D9000323D309D30A5308D9000323FF
:10051000CB2AE2223A3C031DCA2AD301F122D80099
:10052000F1225308031DCA2A203084003C23B03036
:10053000580793008C1D9A2A8C1193008C1D9E2ABB
:100540008C1113088000840A93008C1DA52A8C113D
:1005500013088000840A93008C1DAC2A8C111308A8
:10056000800020308400D3012130E9220008D30725
:10057000D9000323840A0008D307D9000323840A7F
:100580000008D307D9000323840AD309D30A5308E8
:10059000D9000323CB2A08308A00042883120317CA
:1005A0008D00D822831203170C088312031308004E
:1005B0001F308F058316031700308C000C140000C9
:1005C000000008008312031307118C1EE52A1A0885
:1005D0000800831203138718EB2A0C1EED2A9900DA
:1005E000080083120313E222BF3E031C073E0A3EAB
:1005F000D900D90EE222BF3E031C073E0A3ED904B1
:100600005908D307080083120313590E0F39F63E19
:100610000318073E3A3EE92259080F39F63E0318FF
:10062000073E3A3EE9220800831203132430E922F0
:100630007108D9000323D909D90A032308001F3000
:100640008F058316031780308C000C140000000007
:1006500008003C23B23093008C1D2C2B8C1193008E
:100660008C1D302B8C1193008C1D342B8C1193001E
:100670008C1D382B8C11080083120313E11A432BB5
:1006800006150611452B86148610080083120313E5
:100690003C23C03093008C1D4B2B8C11080083121F
:1006A00003133C23503093008C1D542B8C110800F5
:1006B000831203133C23013093008C1D5D2B8C119E
:1006C000080083120313203084003C23B3309300CE
:1006D0008C1D682B8C1193008C1D6C2B8C111308B6
:1006E0008000840A93008C1D732B8C1113088000EA
:1006F000840A93008C1D7A2B8C11130820388000FB
:10070000203084003C23803093008C1D852B8C117D
:10071000000893008C1D8A2B8C11840A000893001A
:100720008C1D902B8C11840A000893008C1D962B35
:100730008C118030073E93008C1D9C2B8C11030183
:1007400093008C1DA12B8C11030193008C1DA62BF3
:0E0750008C11353093008C1DAB2B8C110800E2
:020FFE000102EE
:00000001FF
